:100000000C9436000C945E000C945E000C945E0020
:100010000C945E000C945E000C945E000C945E00E8
:100020000C945E000C945E000C945E000C945E00D8
:100030000C945E000C945E000C945E000C945E00C8
:100040000C942D050C945E000C94D9050C945E0064
:100050000C945E000C945E000C945E000C945E00A8
:100060000C94B1020C945E00A801220711241FBE5B
:10007000CFEFD8E0DEBFCDBF11E0A0E0B1E0E8E314
:10008000F2E102C005900D92A431B107D9F711E059
:10009000A4E1B1E001C01D92A53DB107E1F710E078
:1000A000CCE6D0E004C02297FE010E941609C836B3
:1000B000D107C9F70E9426050C941A090C94000078
:1000C0000F931F93CF93DF93689F8001699F100D5B
:1000D000789F100D1124C8010E947C00EC0100974C
:1000E00029F060E070E0A8010E947E01CE01DF915E
:1000F000CF911F910F910895CF93DF93BC01823070
:10010000910510F462E070E0A091D301B091D401A8
:10011000ED01E0E0F0E040E050E021C0888199810D
:100120008617970769F48A819B81309719F093832A
:10013000828304C09093D4018093D301FE0134C024
:100140006817790738F44115510519F08417950798
:1001500008F4AC01FE018A819B819C01E901209792
:10016000E9F641155105A9F1CA01861B970B0497C1
:1001700008F4BA01E0E0F0E02AC08D919C9111975B
:1001800084179507F9F46417750781F412968D9119
:100190009C911397309719F09383828304C09093B6
:1001A000D4018093D301FD0132964CC0CA01861B55
:1001B000970BFD01E80FF91F6193719302978D93DF
:1001C0009C9340C0FD01828193819C01D9011097CD
:1001D000A1F68091D1019091D201892B41F48091B7
:1001E0000501909106019093D2018093D101409135
:1001F0000701509108014115510541F44DB75EB713
:100200008091030190910401481B590B2091D10169
:100210003091D201CA01821B930B8617970780F099
:10022000AB014E5F5F4F8417950750F0420F531F8D
:100230005093D2014093D101F9016193719302C0AF
:10024000E0E0F0E0CF01DF91CF910895CF93DF930D
:10025000009709F450C0EC0122971B821A82A091EA
:10026000D301B091D401109709F140E050E0AC17F0
:10027000BD0708F1BB83AA83FE0121913191E20FF2
:10028000F31FAE17BF0779F48D919C911197280F3A
:10029000391F2E5F3F4F3983288312968D919C9191
:1002A00013979B838A834115510571F4D093D40130
:1002B000C093D30120C012968D919C911397AD01EC
:1002C000009711F0DC01D3CFFA01D383C2832191CF
:1002D0003191E20FF31FCE17DF0769F4888199810E
:1002E000280F391F2E5F3F4FFA01318320838A8107
:1002F0009B8193838283DF91CF910895DC0101C0BC
:100300006D9341505040E0F7089581E080931D01C6
:100310006093180110921B0110921C0108958091A6
:10032000170190911601891B0895909116018091F3
:100330001701981710F080E00895E0911401F091F2
:100340001501E90FF11D80819F5F909316010895BB
:100350000895DF93CF930F92CDB7DEB76983809175
:100360001D018823A9F080911C018032B0F4809196
:100370001B01E0911901F0911A01E80FF11D608352
:1003800080911B018F5F80931B0180931C0105C02E
:10039000CE01019661E00E9494020F90CF91DF910F
:1003A00008950E94A90108956091190170911A01A0
:1003B0008091180140911C0121E00E944F0210928F
:1003C0001B0110921C0110921D010895862F60914F
:1003D000140170911501413208F040E20E941702A9
:1003E000109216018093170108950E94E601089566
:1003F00080E290E061E070E00E9460008093140170
:1004000090931501109216011092170180E290E06E
:1004100061E070E00E9460008093190190931A01DE
:1004200010921B0110921C010E9433040895982F12
:10043000413210F040E031C080911F018823E1F784
:1004400081E080931F018FEF80933001109227018C
:100450004150409328014F5F990F91609093200184
:1004600085EE8093BC0080911F018130E1F3809183
:100470002701841710F440912701A0912501B09124
:10048000260120E030E007C0FB01E20FF31F8D9151
:1004900080832F5F3F4F2417B8F3842F08951F9355
:1004A000582F122F413210F081E03CC080911F0183
:1004B0008823E1F782E080931F018FEF8093300162
:1004C0001092270140932801A0912501B0912601A7
:1004D000FB0102C081918D938E2F861B8417D0F370
:1004E000852F90E0880F991F8093200185EE8093DF
:1004F000BC00112321F080911F018230E1F3809133
:1005000030018F3F11F480E00DC0809130018032C6
:1005100011F482E007C080913001803311F084E053
:1005200001C083E01F910895482F613210F081E0EF
:10053000089580911F01843011F082E00895609346
:100540002C01A0912901B0912A01842F9C01F9016D
:1005500002C081918D938E2F841B8617D0F380E08B
:1005600008951F920F920FB60F9211242F933F936D
:100570004F935F936F937F938F939F93AF93BF93AB
:10058000EF93FF938091B90090E0887F9070803660
:10059000910509F4E2C081369105CCF588329105C8
:1005A00009F47BC089329105B4F48031910509F4D6
:1005B0006FC0813191053CF4009709F438C1089768
:1005C00009F040C165C08831910509F466C0809783
:1005D00009F038C17FC08034910509F4A3C081348B
:1005E000910544F48033910509F47FC0C89709F060
:1005F00029C186C08035910509F486C088359105EA
:1006000009F495C08834910509F01CC19EC0883951
:10061000910509F404C189399105ECF488379105F5
:1006200009F49BC0893791054CF48836910509F48B
:1006300094C08037910509F005C18FC088389105B5
:1006400009F4EDC08039910509F48DC08038910519
:1006500009F0F8C088C0803B910509F4B2C0813B25
:1006600091054CF4803A910509F491C0883A9105BE
:1006700009F0E8C0A6C0803C910509F4D4C0883CCC
:10068000910509F4D0C0883B910509F0DBC0B1C0E9
:10069000809120018093BB00C0C090912701809180
:1006A0002801981778F490912701E0912501F091A5
:1006B0002601E90FF11D80818093BB009F5F90931D
:1006C0002701ABC085ED8093BC008091BC0084FD08
:1006D000FCCFB6C080E28093300185ED8093BC00F2
:1006E0008091BC0084FDFCCFABC080E380933001DF
:1006F00085ED8093BC008091BC0084FDFCCFA0C040
:1007000088E3809330018FC0809127019091BB00D6
:10071000E0912501F0912601E80FF11D90838F5F94
:1007200080932701909127018091280174C08091C6
:1007300027019091BB00E0912501F0912601E80F7F
:10074000F11D90838F5F8093270185ED8093BC001E
:100750008091BC0084FDFCCF73C083E080931F01B7
:1007600010922F015AC080912F01803208F057C09B
:1007700080912F019091BB00E0912D01F0912E010D
:10078000E80FF11D90838F5F80932F0146C0809109
:100790002F01803248F480912F01E0912D01F091DA
:1007A0002E01E80FF11D108260912F01E0912301CD
:1007B000F091240180912D0190912E0170E0099516
:1007C00032C084E080931F0110922B0110922C0103
:1007D000E0912101F0912201099580912C0188235B
:1007E00041F481E080932C01E0912901F0912A01EC
:1007F000108290912B01E0912901F0912A01E90FDB
:10080000F11D80818093BB009F5F90932B0190919D
:100810002B0180912C01981710F485EC01C085E81C
:100820008093BC000FC085EC8093BC0009C010927F
:10083000300185ED8093BC008091BC0084FDFCCF2D
:1008400010921F01FF91EF91BF91AF919F918F91F6
:100850007F916F915F914F913F912F910F900FBEBC
:100860000F901F90189510921F01449A459AE9EB3A
:10087000F0E080818E7F808380818D7F808388E41B
:100880008093B80085E48093BC0080E290E061E052
:1008900070E00E946000809325019093260180E221
:1008A00090E061E070E00E946000809329019093E5
:1008B0002A0180E290E061E070E00E946000809395
:1008C0002D0190932E0108950F931F93082F8EE111
:1008D00091E06DE170E00E948501112707FD109500
:1008E0008EE191E0B8010E94D1018EE191E00E9479
:1008F000D4018EE191E06DE170E041E050E00E94B2
:10090000F5018EE191E00E948F01882329F08EE1AC
:1009100091E00E94950100C01F910F9108950F93DF
:100920001F93883739F482E30E946404082F10E093
:1009300083E311C0893739F484E30E946404082FEB
:1009400010E085E308C08A3761F486E30E946404FE
:10095000082F10E087E30E946404382F20E0200F66
:10096000311FC9011F910F910895EF92FF920F93CC
:100970001F9388E70E948F040EEB11E0AC016627FD
:1009800057FD6095762FC8012AE030E00E947C0870
:1009900080E0E82E81E0F82EC801B7010E9493079D
:1009A00089E70E948F04AC01662757FD6095762F7A
:1009B000C8012AE030E00E947C08C801B7010E940B
:1009C00093078AE70E948F04AC01662757FD609564
:1009D000762FC8012AE030E00E947C08C801B701E8
:1009E0000E949307C80162E071E00E94B2076CE2C6
:1009F00071E080E090E00E9475051F910F91FF90DB
:100A0000EF9008950F931F930EE111E0C8010E942B
:100A1000F8018EEB91E040E05BE460E070E00E9462
:100A20001606C8016DE170E00E948501C8016DE203
:100A300070E00E94D101C80169E070E00E94D1011C
:100A4000C8010E94D4011F910F9108950E949F0533
:100A50000E9402050E94B504FDCF1F920F920FB6AF
:100A60000F9211242F933F938F939F93AF93BF9334
:100A70008091350190913601A0913701B0913801F4
:100A8000309139010196A11DB11D232F2D5F2D3706
:100A900020F02D570196A11DB11D2093390180939F
:100AA000350190933601A0933701B09338018091BE
:100AB000310190913201A0913301B091340101963E
:100AC000A11DB11D8093310190933201A093330198
:100AD000B0933401BF91AF919F918F913F912F912E
:100AE0000F900FBE0F901F901895EF92FF920F93EB
:100AF0001F937B018C018FB7F89440913501509181
:100B0000360160913701709138018FBF2FB7F8948B
:100B10008091350190913601A0913701B091380153
:100B20002FBF841B950BA60BB70BE816F9060A0717
:100B30001B0760F71F910F91FF90EF900895789435
:100B400084B5826084BD84B5816084BD85B58260D2
:100B500085BD85B5816085BDEEE6F0E08081816070
:100B60008083E1E8F0E08081826080838081816021
:100B70008083E0E8F0E0808181608083E1EBF0E059
:100B8000808184608083E0EBF0E0808181608083FD
:100B9000EAE7F0E0808184608083808182608083E6
:100BA0008081816080838081806880831092C10011
:100BB00008951F920F920FB60F9211242F933F9317
:100BC0004F935F936F937F938F939F93AF93BF9355
:100BD000EF93FF934091C600E091BA01F091BB0101
:100BE000CF01019660E870E00E94B0089C018091FE
:100BF000BC019091BD012817390739F0E65CFE4F22
:100C000040833093BB012093BA01FF91EF91BF91D4
:100C1000AF919F918F917F916F915F914F913F9194
:100C20002F910F900FBE0F901F9018955F926F92AB
:100C30007F928F929F92AF92BF92CF92DF92EF926C
:100C4000FF920F931F93CF93DF93EC013A014B0177
:100C5000413482E458078FE0680780E078070CF0A1
:100C60007FC060E874E88EE190E0A40193010E94E7
:100C7000E5082150304040405040CA01B90122E00F
:100C800030E040E050E00E94E50859016A01A60109
:100C90009501209530954095509594E0220F331F93
:100CA000441F551F9A95D1F760E074E284EF90E0FD
:100CB0000E94E508CA01B9012FEF30E040E050E0A2
:100CC0000E949108A40193010E94E508C901815086
:100CD0009F4F181619061CF4522E5A9403C055241F
:100CE0005394521A60E079E08DE390E0A4019301FF
:100CF0000E94E5082150304040405040CA01B901EF
:100D000022E030E040E050E00E94E5082095309578
:100D10004095509583E0220F331F441F551F8A953D
:100D2000D1F760E074E284EF90E00E94E508CA0128
:100D3000B9012FEF30E040E050E00E949108A4019B
:100D400093010E94E508C90181509F4F18161906AA
:100D50001CF4822F815002C081E0821B851500F5B2
:100D6000E885F98581E090E00A8802C0880F991F24
:100D70000A94E2F7808360E079E08DE390E0A401DB
:100D800093010E94E5082150304040405040CA0184
:100D9000B90122E030E040E050E00E94E50804C0E4
:100DA000E885F98510829501EC81FD813083EE8123
:100DB000FF812083EA85FB85208141E050E0CA0164
:100DC0000E8402C0880F991F0A94E2F7282B208313
:100DD000EA85FB852081CA010F8402C0880F991F14
:100DE0000A94E2F7282B2083EA85FB858081088816
:100DF00002C0440F551F0A94E2F7842B8083DF91D1
:100E0000CF911F910F91FF90EF90DF90CF90BF9007
:100E1000AF909F908F907F906F905F900895FC01AE
:100E2000A085B18521898C9190E0022E02C0959514
:100E300087950A94E2F780FFF6CF0484F585E02DCC
:100E4000608308958DE091E09093BF018093BE018F
:100E50008AE391E09093C1018093C00185EC90E01A
:100E60009093C3018093C20184EC90E09093C501FC
:100E70008093C40180EC90E09093C7018093C601F9
:100E800081EC90E09093C9018093C80186EC90E0DA
:100E90009093CB018093CA0184E08093CC0183E0DE
:100EA0008093CD0187E08093CE0185E08093CF01D0
:100EB00081E08093D00108950F931F93CF93DF9328
:100EC0008C01EB0109C02196D801ED91FC910190B4
:100ED000F081E02DC801099568816623A1F7DF91B3
:100EE000CF911F910F910895EF92FF920F931F934F
:100EF000CF93DF938C017B01EA010CC0D7016D9188
:100F00007D01D801ED91FC910190F081E02DC801A7
:100F100009952197209791F7DF91CF911F910F911C
:100F2000FF90EF900895DC01ED91FC910280F38138
:100F3000E02D099508950F931F938C01DC01ED912D
:100F4000FC910190F081E02D6DE00995D801ED91C3
:100F5000FC910190F081E02DC8016AE009951F9194
:100F60000F9108950F931F938C010E949307C8015E
:100F70000E949B071F910F9108952F923F924F92CD
:100F80005F926F927F928F929F92AF92BF92CF9219
:100F9000DF92EF92FF920F931F93DF93CF93CDB722
:100FA000DEB7A0970FB6F894DEBF0FBECDBF1C0111
:100FB0006A017B01411551056105710549F4DC01A8
:100FC000ED91FC910190F081E02D60E3099554C012
:100FD000882499245401422E55246624772401E064
:100FE00010E00C0F1D1F080D191DC701B601A3014C
:100FF00092010E94C308F80160830894811C911C2F
:10100000A11CB11CC701B601A30192010E94C30833
:10101000C901DA016C017D01C114D104E104F104BC
:10102000F1F681E0E82EF12CEC0EFD1EE80CF91C27
:101030003E010894611C711CD501C4010197A109EE
:10104000B1096C01C818D90814C0F601EE0DFF1DD6
:1010500060816A3010F4605D01C0695CD101ED917E
:10106000FC910190F081E02DC10109950894E108FF
:10107000F1086E147F0449F7A0960FB6F894DEBF0E
:101080000FBECDBFCF91DF911F910F91FF90EF90D9
:10109000DF90CF90BF90AF909F908F907F906F9098
:1010A0005F904F903F902F900895EF92FF920F9393
:1010B0001F93CF93DF93EC017A018B0177FF0FC071
:1010C000E881F9810190F081E02D6DE2099510959C
:1010D0000095F094E094E11CF11C011D111DCE015E
:1010E000B801A7012AE00E94BD07DF91CF911F91AF
:1010F0000F91FF90EF900895DC012115310541F427
:10110000ED91FC910190F081E02D642F09950895F7
:101110002A30310519F40E94550808950E94BD0730
:101120000895629FD001739FF001829FE00DF11D31
:10113000649FE00DF11D929FF00D839FF00D749F51
:10114000F00D659FF00D9927729FB00DE11DF91FFD
:10115000639FB00DE11DF91FBD01CF01112408955A
:1011600097FB092E07260AD077FD04D049D006D078
:1011700000201AF4709561957F4F0895F6F79095C9
:1011800081959F4F0895A1E21A2EAA1BBB1BFD015A
:101190000DC0AA1FBB1FEE1FFF1FA217B307E40756
:1011A000F50720F0A21BB30BE40BF50B661F771FAE
:1011B000881F991F1A9469F760957095809590958E
:1011C0009B01AC01BD01CF01089597FB092E0526B7
:1011D0000ED057FD04D0D7DF0AD0001C38F450954C
:1011E0004095309521953F4F4F4F5F4F0895F6F74B
:1011F00090958095709561957F4F8F4F9F4F089583
:10120000AA1BBB1B51E107C0AA1FBB1FA617B7072C
:1012100010F0A61BB70B881F991F5A95A9F7809548
:101220009095BC01CD010895EE0FFF1F0590F4913C
:08123000E02D0994F894FFCFB2
:101238007400002000D5010000000000000F075CCA
:041248000774070020
:00000001FF
